:100000000C943F030C945C030C945C030C945C0311
:100010000C945C030C945C030C945C030C945C03E4
:100020000C945C030C945C030C948E130C94D0120F
:100030000C941A1D0C945C030C945C030C945C03EC
:100040000C945C030C945C030C945C030C945C03B4
:100050000C945C030C9419150C945C030C945C03D5
:100060000C945C030C945C030C945C030C945C0394
:100070000C945C030C945C030C945C030C945C0384
:100080000C945C030C945C030C945C030C945C0374
:100090000C945C030C945C030C945C030C945C0364
:1000A0000C945C030C945C030C945C0308067C06C3
:1000B0001006DA05DE051406E10517062206EC0532
:1000C0007206F0052606F4052A065406F8052E06E3
:1000D0005E06FE0534063E06E5051B06E8051E061F
:1000E000030639064A066A066C06D6050C0685061E
:1000F000AE06B4069F06A506BA06C006C606700779
:100100007007A307A3071D083B08430943094008DC
:10011000B408C508C5088609A209A709AC09B10930
:10012000B609BB09C009C509CA09CF09D609D90949
:10013000DC09DF09E209E509E809EB09EE09F30941
:100140009F0DA20DC70DEA0DF20DFD0D000E000E64
:10015000000E130F130F7A0E7C0E810EA70ECA0E1F
:10016000CD0ED00EF30EE8100F11B8120F11B81209
:100170005B117E11B81273128312000000000000A0
:10018000000000000000000000000000000000006F
:1001900000000000000000000000000000007E0FD2
:1001A00000D4FFFFFFC7000000780000000000003F
:1001B00000002A2B280000000000000000000000C2
:1001C000000000000029000000002C1E3420212225
:1001D00024342627252E362D3738271E1F2021228E
:1001E000232425263333362E37381F040506070807
:1001F000090A0B0C0D0E0F101112131415161718F7
:10020000191A1B1C1D2F3130232D35040506070834
:10021000090A0B0C0D0E0F101112131415161718D6
:10022000191A1B1C1D2F3130354C1E0F0500047F81
:100230003F1F643214643214783C1E1E140A0505F4
:10024000010902A10185020901A10005091901297D
:10025000081500250195087501810205010930097D
:10026000311581257F95027508810609381581258C
:100270007F950175088106050C0A38021581257FD6
:10028000950175088106C0C005010980A10185039B
:1002900019012AB700150126B700950175108100D4
:1002A000C0050C0901A101850419012AA00215014C
:1002B00026A002950175108100C005010906A10163
:1002C0008506050719E029E7150025019508750140
:1002D00081020507190029EF1500250195F0750128
:1002E00081020508190129059505750191029501FD
:1002F00075039101C00660FF0961A1010962150043
:1003000026FF009520750881020963150026FF006D
:10031000952075089102C005010906A1010507197C
:10032000E029E71500250195087501810295017501
:100330000881010507190029FF150026FF00950611
:1003400075088100050819012905950575019102B7
:10035000950175039101C009025B00030100A0FA39
:10036000090400000103010100092111010001221B
:100370004000070581030800010904010002030091
:10038000000009211101000122220007058203203B
:100390000001070503032000010904020001030016
:1003A000000009211101000122B600070584032085
:1003B00000011201000200000008756F61010100D8
:1003C000010200011003530077006500650074000E
:1003D0003100360000001C03310075007000200061
:1003E0004B006500790062006F00610072006400DC
:1003F00073000000040309042223252628292A2C3F
:100400002D2F3032333536383A3B3D3E404243455E
:1004100047494A4C4E5051535557595A5C5E606299
:10042000646668696B6D6F71737577797B7D7F81A9
:10043000838587898A8C8E90929496989A9C9E9FA9
:10044000A1A3A5A7A8AAACAEAFB1B3B4B6B8B9BBC7
:10045000BCBEBFC1C2C3C5C6C7C9CACBCCCDCED036
:10046000D1D2D2D3D4D5D6D7D7D8D9D9DADADBDB23
:10047000DBDCDCDCDCDCDDDDDDDDDCDCDCDCDCDBBA
:10048000DBDBDADAD9D9D8D7D7D6D5D4D3D2D2D103
:10049000D0CECDCCCBCAC9C7C6C5C3C2C1BFBEBCF6
:1004A000BBB9B8B6B4B3B1AFAEACAAA8A7A5A3A167
:1004B0009F9E9C9A98969492908E8C8A8987858329
:1004C000817F7D7B79777573716F6D6B6968666409
:1004D00062605E5C5A5957555351504E4C4A4947D9
:1004E000454342403E3D3B3A3836353332302F2D7E
:1004F0002C2A29282625232224002500260025022F
:1005000021002200230038001E001F0020002D00C3
:100510002700280037002152007C01000100010063
:1005200001000100010001000100010001000100C3
:1005300001000100010001000100010001000100B3
:1005400001000100010001000100010001000100A3
:100550000100010001000100010001000100010093
:100560000100010001000100010001000100010083
:100570000100010001000100000101010101010170
:100580000101020202020202020202030303030348
:100590000303030404040404040405050505050617
:1005A00006060606070707070708080808090909D5
:1005B000090A0A0A0B0B0B0C0C0C0D0D0D0E0E0E7E
:1005C0000F0F0F101011111112121313141415150F
:1005D00016161717181819191A1A1B1B1C1D1D1E81
:1005E0001E1F2020212222232424252626272829D5
:1005F000292A2B2C2D2D2E2F303132323334353603
:100600003738393A3B3C3D3E3F4041424344454602
:100610004748494A4C4D4E4F5051535455565859DE
:100620005A5B5D5E5F616264656668696B6C6D6F85
:100630007072737577787A7B7D7E808283858788F8
:100640008A8C8E8F91939596989A9C9EA0A2A3A532
:10065000A7A9ABADAFB1B3B5B7BABCBEC0C2C4C633
:10066000C9CBCDCFD1D4D6D8DBDDDFE2E4E7E9EBEF
:10067000EEF0F3F5F8FAFDFFFFAA7F5540001124D4
:100680001FBECFEFDAE0DEBFCDBF11E0A0E0B1E0EA
:10069000E8E0FEE402C005900D92A239B107D9F757
:1006A00022E0A2E9B1E001C01D92A139B207E1F751
:1006B0000E94FE090C9402270C9400000E945D2009
:1006C0002FEF84E39CE0215080409040E1F700C090
:1006D00000009AE088E10FB6F894A8958093600036
:1006E0000FBE90936000FFCFA7E1B0E0EAE7F3E030
:1006F0000C94C0264B8B5C8B6D8B7E8B8F8B61112A
:100700001092550286E09E01235F3F4FD901E82FEA
:100710001D92EA95E9F795E0FE017396D9010190E3
:100720000D929A95E1F79C894E895F897B897D8737
:100730009E876F87598B488BF901DE0117960190D0
:100740000D928A95E1F7CE0107960E9480198111DA
:100750003EC086E0FE013796DE01119601900D92B3
:100760008A95E1F7FF81E8856A857B8561157105CA
:1007700031F0EF3F31F481E0FF3F19F403C081E035
:1007800001C080E080FD23C02091020230E0C90159
:100790000196877099274091330250E0841795079E
:1007A00079F1F983EA837D836C8396E0929FD0018F
:1007B000939FB00D1124AD5FBD4FFE0131960190A6
:1007C0000D929A95E1F7809302020E940D1916E0AE
:1007D00080913302909102028917F9F0189FC001AD
:1007E00011248D5F9D4F0E9480198823B1F0809164
:1007F000330290E001968770992780933302E8CF07
:100800000E945D201092020210923302ECEFF1E0A0
:1008100086E0DF011D928A95E9F76796E3E00C9484
:10082000DC26809580FF02C0289A01C0289881FFAD
:1008300002C05D9A08955D980895ADE0B0E0E3E2EE
:10084000F4E00C94B126FC018081918123813481F4
:10085000232B31F09F3F31F491E08F3F19F403C017
:1008600091E001C090E090FDC5C57F0185E0DE010B
:10087000199601900D928A95E1F7F70122818985F9
:100880009A85222349F00E94621F182F682F8985BC
:100890009A850E94D21F03C00E949E1F182F69854F
:1008A0007A85812F0E945D168C01F7018281882351
:1008B00009F42BC19801225037472031310508F047
:1008C00040C18FEF93E00E94B625811128C10250EC
:1008D00036EAA32EB12C002379F0A114F4E0BF0670
:1008E00009F41DC1C5010E94B625811101C0015046
:1008F0002FEFA21AB20AEFCFCE0101962C0188E0A9
:10090000F20111928A95E9F72AE0322E85010F5FF4
:100910001F4FC5010E94B62589831A82882309F4D6
:10092000FEC0813009F041C06501F2E0CF0ED11C5C
:10093000C8010E94B6258A83882309F4F0C09FEF7E
:10094000980F933060F423E0A20EB11CC6010E9400
:10095000B6258B83882309F4E2C01C8229C0843029
:1009600031F54E0133E0830E911C02E010E0560198
:100970008FEFA81AB80AC6010E94B625F401819328
:100980004F01882309F4CBC08C3741F4E2E0F0E05A
:10099000EC0FFD1FE00FF11F10820AC00F5F1F4F09
:1009A00065010730110519F7BAC0580101C0560199
:1009B0008201F8012081222309F4A8CF213009F017
:1009C0004CC08181813049F46801F2E0CF0ED11C26
:1009D000F80182810E949D220AC0823051F4680190
:1009E000F2E0CF0ED11CF80182810E94D92186014C
:1009F00089C0833049F46801F2E0CF0ED11CF801C0
:100A000082810E947521F3CF843019F00F5F1F4F50
:100A100079C0F80122810E5F1F4F80E090E030E046
:100A2000205331092A30310568F4389EA001399EDF
:100A3000500D1124C901840F951F0F5F1F4FF8013E
:100A40002081EDCF009709F45DC0EFE9FFE0319719
:100A5000F1F700C000000197F5CFE22FF0E0E65576
:100A6000FE4F2490822F86958695869590E0FC0116
:100A7000E656FE4F64902770712C022E02C07594CA
:100A800067940A94E2F7F1E06F227724FC01E657BD
:100A9000FE4F8490912C022E02C0959487940A9464
:100AA000E2F731E083229924FC01E658FE4FC4901E
:100AB000D12C02C0D594C7942A95E2F781E0C822D0
:100AC000DD246114710419F081EE0E94D921811492
:100AD000910419F086EE0E94D921822D0E949D2258
:100AE0008114910419F086EE0E947521611471043D
:100AF00019F081EE0E947521C114D10419F08CE225
:100B00000E949D220F5F1F4F54CF011537E7130737
:100B100009F042C181E00E940A200E94F90F8091F1
:100B20003402877009F466C4F7018281882309F4CE
:100B300061C48091AB0182FF5DC482E00E94D9183C
:100B400059C40115F7E71F0711F481E005C0013012
:100B500027E7120721F482E00E941720DECFF80178
:100B6000E851FC47E730F10508F4E5C0882309F4B3
:100B70005BC110926E02C8019057839708F013C1B1
:100B800084E090E00E94C4259093AB018093AA0179
:100B9000F801E150F047E232F10520F4EA5AFF4F44
:100BA0000C9495268091AA018160ACC08091AB0124
:100BB0008860B4C08091AA018260A4C08091AA011B
:100BC00020C08091AA0188609DC08091AB011EC0A9
:100BD0008091AB018260A2C08091AA01806192C025
:100BE0008091AA0180628EC08091AA0180648AC02F
:100BF0000E945D208091AA01806884C08091AA0132
:100C0000886084607FC08091AB018260816086C013
:100C10008091AA018E7F76C08091AB01877F7EC0D4
:100C20008091AA018D7F6EC08091AA0120C0809121
:100C3000AA01877F67C08091AB011EC08091AB0184
:100C40008D7F6CC08091AA018F7E5CC08091AA01CB
:100C50008F7D58C08091AA018F7B54C00E945D2077
:100C60008091AA018F774EC08091AA01877F8B7FE8
:100C700049C08091AB018D7F8E7F50C08091AA01C9
:100C800082FB222720F991E0922790FB82F990FBCA
:100C900083F938C08091AB01982F909591708E7F29
:100CA000892B90FB81F93AC08091AA0186FB22270B
:100CB00020F991E0922790FB86F924C00E945D20E4
:100CC0008091AA0187FB222720F991E0922790FBCF
:100CD00087F918C061E001C060E08EE090E00E94FA
:100CE000CA251EC08091AA0184FB222720F991E029
:100CF000922790FB84F906C08091AA01982F9095C5
:100D000090FB80F98093AA010BC08091AB0183FB1B
:100D1000222720F991E0922790FB83F98093AB0181
:100D20006091AA017091AB0184E090E00E94E825F7
:100D30000E945D20F4CEE858FF4F0C94952606E201
:100D400021EE41EE6AE17CE705C007E225EE45EEC3
:100D50006BE17CE7C7010E94F71DE1CE06E221EEC0
:100D600040EE68E17CE7F6CF07E225EE44EE69E16C
:100D70007CE7F0CF06E221EE42EE6CE17CE7EACFC1
:100D800007E225EE46EE6DE17CE7E4CF08E221E0E4
:100D900045EE6EE17CE7DECF013097E7190709F0F9
:100DA000DECE82E0B8CE0631ECE71E0709F48CC235
:100DB00003309CE7190721F140F40115FCE71F07F8
:100DC00089F001301C4711F13EC00B353CE7130799
:100DD00039F10C358CE71807D9F00A351C4799F51D
:100DE00081E01FC00E945D20EFEFF4E32CE0E150B2
:100DF000F0402040E1F700C000000E9408158FCEAF
:100E00006FEF7FEF80E090E00E94E8250E945E0394
:100E10008091AB0182FB882780F991E0892701C08E
:100E200080E00E94F6180FC00631FCE71F0709F4A6
:100E30005BC2809156028272F801E052F847E531B8
:100E4000F10508F45FC2F7018281008111818823D6
:100E500049F0C8010E94621FD82E682FC8010E9465
:100E6000D21F04C0C8010E949E1FD82EB8018D2D2C
:100E70000E945D160E946B16B82E192F982EF7014E
:100E80000281A580A2949FE0A922809134028770FC
:100E9000B9F00023A9F0812F807F803421F080E217
:100EA0008B0D883068F08091AB0182FF09C082E031
:100EB0000E94D918809134028770DD24D394811167
:100EC000D12CC12EC2948FE0C8228C2D90E08C30A2
:100ED000910508F0D8C1FC01E158FF4F0C9495260C
:100EE000812F807F1F70882311F01295107F0023BF
:100EF000B9F0112309F4B5C180E28B0D883010F0F0
:100F0000911006C090915602192B1093560205C0FD
:100F100090915502192B109355020E948418A1C17B
:100F20008B2D0E947521112309F4ADC180E28B0D38
:100F3000883088F1992079F1109590915502192304
:100F4000109355022BC0812F807F1F70803211F0CB
:100F50001295107F8B2D992029F0F1E09F1609F44E
:100F600041C04FC08091AB0182FD1BC0002369F0DE
:100F7000112339F090915602192B109356020E94BA
:100F8000841880E00E94D9217EC180E00E947521F2
:100F9000112309F478C1812F0E947D180E948418C2
:100FA00072C1002381F080915702AA2051F021E004
:100FB000A21207C0182B181709F465C11093570225
:100FC00062C1812B16C0A11003C00E94771831C0E6
:100FD00031E0A31609F457C1812F0E948C200E9492
:100FE000771851C1002341F085E08A1508F44BC100
:100FF000812F0E94932047C194E09A1508F443C1C1
:1010000018C0002349F0AA2099F3F701858180FFD9
:1010100028C18F708583ECCFAA2059F0893309F05D
:101020002FC1FFEF27EE33E0F15020403040E1F7D1
:1010300025C1812F0E948C2026C1812F86958695FF
:10104000837019F0813061F01EC1002321F08B2DD7
:10105000912F937002C080E090E00E94C51D1BC1DB
:10106000002321F08B2D912F937002C080E090E03F
:101070000E94A01D10C1602F8B2D0E949D200BC1CE
:10108000812F8370A9F5011102C14B2D4295469520
:101090004770440F440F8B2D8F7090E09C01042EFD
:1010A00001C0220F0A94EAF7B4FE08C08FE090E076
:1010B00001C0880F4A95EAF7809501C080E0169537
:1010C00016951370123069F088F49091580211301F
:1010D00019F0822B892302C0922B892B0E94232096
:1010E000D6C0822B909158028927F8CF822BF6CF59
:1010F000002319F0812F817001C08695882309F49F
:10110000C6C04B2D429546954770440F440F8B2D1A
:101110008F7090E09C01042E01C0220F0A94EAF720
:10112000B4FE08C08FE090E001C0880F4A95EAF74E
:10113000809501C080E0169516951370123059F015
:1011400078F49091DB01113019F0822B892309C0CA
:10115000922B892B06C0822B9091DB01892701C03D
:10116000822B0E94072093C01F70002339F0812F2B
:101170000E9417208B2D0E94932089C08B2D0E94E6
:101180008C20812F0E940A2082C08B2D92EF99160D
:1011900081F1991538F0E0EF9E1659F0F1EF9F16A6
:1011A00019F15BC023EF921659F134EF9316C1F099
:1011B00054C0002381F084E08A1508F464C01F71D4
:1011C00081E090E0012E01C0880F0A94EAF7909127
:1011D000DB01892720C095E09A1508F454C0EFCFB1
:1011E0008091AB0182FD1AC0002329F0812F8F71FD
:1011F00027C00023D9F3812F8F710E940A2043C09A
:10120000002341F01F7181E0012E01C0880F0A9474
:10121000EAF701C080E00E94072035C0002399F062
:101220001F71812F0E9417208091AB0182FF07C0A0
:10123000E8E01E9FC0011124836080933402812F57
:101240000E94172020C081E00E94D918F1E0FA1511
:10125000D0F482E00E94D91816C0002321F0AA2001
:1012600029F28B2D8FCEAA2031F2893349F42FEF4A
:1012700037EE83E0215030408040E1F700C00000AD
:101280008B2D0E94752188EF8C0D843020F40E94F4
:10129000EA1D0E941104DD2009F4ACC080913402E3
:1012A00080FDA8C0F70112828595859585950E94DD
:1012B0001720C7010E941D048091340285958595F1
:1012C00085950E940A2096C0809156028A7A91E004
:1012D00009F490E090939401811112C069E28CEDC1
:1012E00091E00E946B1D09C080919401811180C022
:1012F00069E28CED91E00E94431D0E9484180FCC9E
:1013000065E3EDCFE557FF4F0C949526809167027A
:1013100080FF12C08E7F8093670260916702709198
:1013200068028091690290916A020E940D231092D6
:1013300090020E94BC22F3CB81608093670261E03F
:1013400086954EC049ED54E263EE74E22CC043EE44
:1013500054E269ED74E227C043E854E26DE874E2B8
:1013600022C04DE854E263E874E21DC049E654E24D
:1013700066E774E218C046E754E269E674E213C017
:101380004FE454E26CE574E20EC04CE554E26FE4C5
:1013900074E209C040E253E262E373E204C042E354
:1013A00053E260E273E20E945B1FB9CB61E081E02F
:1013B00017C065E082E019C068E086E016C06EE004
:1013C00089E013C064E18FE010C067E185E10DC0E2
:1013D00061E088E105C062E289E107C061E083E283
:1013E0000E9497249CCB6AE285E20E94471F97CB1C
:1013F00065E37FCF2D96E2E10C94CD26AAE2B0E022
:10140000E4E0FAE00C94B12685B7806885BF85B723
:10141000806885BF84B7877F84BF0FB6F894A8958E
:1014200080916000886180936000109260000FBE20
:1014300090E080E80FB6F89480936100909361008B
:101440000FBE8EE495E190939301809392010E94E8
:1014500014130E9433138091E20084608093E200B1
:1014600078948091D1018823A1F01091E9001F7038
:101470009091EC00892F817090FD80E8182B1092DC
:10148000E9008091E80083FD0E9405101F70109311
:10149000E90082E084BD93E095BD9AEF97BD80930B
:1014A0006E000E942E1F811102C00E941E1F0BE1C0
:1014B00011E0D8018D918D018F3F11F00E9493159D
:1014C000B1E00F311B07A9F70FE111E0F80181919D
:1014D0008F018F3F11F00E949315F1E003321F0737
:1014E000A9F784E0E2EAF1E0DF01282F1D922A95B6
:1014F000E9F7E5E9F1E0DF011D928A95E9F70E943D
:101500000918811102C00E94151882E090E00E9423
:10151000B62580939C0184E090E00E94C4259093BE
:10152000AB018093AA010E94AA15EFE3FCE9319771
:10153000F1F700C000000E94AA158091A20180FF6F
:1015400008C06FEF7FEF80E090E00E94E8250E94E6
:10155000081583E090E00E94B6250E942320209A7F
:10156000289A559A5D9A80919901811133C00E9401
:101570000918811104C00E9415180E94442388E0B4
:1015800090E00E94BE25609367027093680280938A
:10159000690290936A026E7F71F40E94442388E08E
:1015A00090E00E94BE25609367027093680280936A
:1015B000690290936A020E94FA221092900280912E
:1015C000670280FF04C060E086950E94972481E056
:1015D0008093990184E091E090937202809371026C
:1015E00068E1462E512C71EAC72E71E0D72EBB243C
:1015F000B3948E010F5F1F4F8091D101853009F0A8
:1016000049C040E1E42E52E1F52E8091D1018530B0
:1016100009F03AC08091D101843029F180E00E9424
:10162000110410927502F0E40FB6F894A895409258
:1016300060000FBEF093600083B7817F846083BF3A
:1016400083B7816083BF7894889583B78E7F83BF8B
:101650000FB6F894A895809160008861809360002F
:10166000109260000FBE8091D001882309F4CDCF85
:101670000E94AA15E2EAF1E081918111DDC321E027
:10168000E63AF207C9F7C1CF0E945D200E94EA1D29
:101690000E9411040E94AA152DE9822E21E0922EAB
:1016A00032EAE32E31E0F32ED701F40191918D91CE
:1016B0008927CE16DF0619F08823C1F322C08111D5
:1016C00020C00E940E1D7C0180919A0190919B0187
:1016D000E816F90609F447C08FEF89A38AA31BA275
:1016E0000E940E1D8160782F9DA38CA349A15AA151
:1016F0006BA18DA10E947403F0929B01E0929A016C
:1017000032C0712CD7012D907D01F401308032243C
:1017100009F1612CAA24A394832D8A21A1F06EA241
:101720007FA291E0822D8A2109F490E098A70E947F
:101730000E1D8160782F9AA789A74EA15FA168A589
:101740008AA50E9474036394AA0CF4E06F12E4CF9C
:10175000D4012C927394BFEF8B1A9B0AE4E07E12A3
:10176000D1CF0E94021D80919002882309F4AAC063
:1017700080918F02E0916702E695E81BE0938B026F
:10178000823059F4F0E0E55CFD4FE491EE2EF12C4F
:101790009EEE892E9CE1992E70C0863059F4F0E0BF
:1017A000E85CFD4FE491EE2EF12C8EED882E8CE15D
:1017B000982E63C0893061F4E695F0E0EB5CFD4F54
:1017C000E491EE2EF12CBBE88B2EBCE19B2E55C094
:1017D0008F3061F4E695F0E0EE5CFD4FE491EE2E83
:1017E000F12CA5E48A2EACE19A2E47C0853159F43C
:1017F000F0E0E15DFD4FE491EE2EF12CF7E18F2E4C
:10180000FCE19F2E3AC08831F9F0833249F4EDE2D1
:10181000F2E0E590F490E4EA8E2EECE19E2E2DC0ED
:101820008432D1F0853209F58E2F63E00E94612663
:10183000E92FF0E0E65DFD4FE491EE2EF12C78E02B
:10184000872E7BE1972E19C058E2E52EF12C60EB34
:10185000862E6BE1962E11C034EFE32EFF24F39415
:1018600043E9842E4BE1942E08C090EDE92E97E0D9
:10187000F92E27E0822E2BE1922E80918C02882374
:1018800061F010928C020E940E1D90938A02809348
:10189000890210928E0210928D020E940E1DE0911C
:1018A0008902F0918A028E1B9F0B8F3F9F4750F455
:1018B000EE0EFF1EF0928A02E092890289E892E021
:1018C000F401099586E0E3E8F2E0D80101900D9279
:1018D0008A95E1F710928502109286021092870293
:1018E000109288028B81811104C08C81882309F4B5
:1018F00051C080918102909182020E943F159C010B
:1019000090917C02992309F4B5C22531310508F480
:1019100041C09F3F19F09F5F90937C02FB80FF20A6
:1019200061F00E943A251F1414F491E001C09FEF6A
:10193000899F802D112480938502FC80FF2061F017
:101940000E943A251F1414F491E001C09FEF899F73
:10195000802D112480938602309185023323D1F0AB
:10196000209186022223B1F045EB3403C0011124FB
:10197000992319F09093850202C0B092850235EB4D
:101980002303C0011124992319F09093860202C009
:10199000B09286028D81811104C08E81882309F462
:1019A00051C080917F02909180020E943F159C015E
:1019B00090917D02992309F462C22135310508F422
:1019C00041C09F3F19F09F5F90937D02FD80FF20F3
:1019D00061F00E9418251F1414F491E001C09FEFDC
:1019E000899F802D112480938702FE80FF2061F063
:1019F0000E9418251F1414F491E001C09FEF899FE5
:101A0000802D112480938802309187023323D1F0F6
:101A1000209188022223B1F045EB3403C001112448
:101A2000992319F09093870202C0B092870235EB98
:101A30002303C0011124992319F09093880202C056
:101A4000B092880246E050E0B80183E892E00E943C
:101A5000F526892BA9F48091850281110FC0809110
:101A6000860281110BC080918702811107C081E03D
:101A700090918802911103C080E001C081E080FD57
:101A80000E94EE2486E0F801A3E8B2E001900D92F6
:101A90008A95E1F70E94EA1DF82E8091A101F816BF
:101AA00039F0F092A1010E94021D8F2D0E941104B5
:101AB0008091D101843009F09FCD83E08093E900CB
:101AC0008091E80082FF98CD8091E80085FF21C0D9
:101AD0000E94651481111BC080E2882E912C780130
:101AE00009C08091F100D7018D937D01B1E08B1A7F
:101AF000910869F08091E80085FDF3CF8091E800BE
:101B00008B778093E8000E946514882399F391E015
:101B100001C090E08091E8008B778093E8009923E2
:101B200009F46ACD2981822F90E0FC013197E331DD
:101B3000F10508F078C1E056FF4F0C9495261A8203
:101B40008BE0DDC08A81823009F48CC150F4813091
:101B500009F069C10E94021D9B838C837D836E8383
:101B600064C1833041F0843009F05DC11B821C8266
:101B70001D821E825AC18091A2018B838091A30194
:101B80008C838091A4018D838091A50129C08A81D5
:101B9000823019F0853051F046C16B817C818D8196
:101BA0009E810E949B260E94FA1E3FC1809167027F
:101BB00080FF0AC0809167028E7F80936702109237
:101BC00090020E94BC2231C181608093670260E074
:101BD000869550C04C816B818A810E94CC1E9D836A
:101BE0008E8323C12D813E813227232732274C81CA
:101BF0006B818A810E94701E18C10E94971E15C1B8
:101C00008A81823009F00FC12830F1F1293009F4BE
:101C100066C08B818230F9F098F4813009F005C1FB
:101C20008C81EFEF8E9FC00111246FEF70E00E9456
:101C30006D26462F20E0609169028091680221C0E4
:101C40008330D9F0843009F0F0C020E040916A027E
:101C50006D818C8116C08C81882309F4ABCF809173
:101C6000670281608093670260E086950E949724F6
:101C700060E08C810E949724D8C08C8180936B0295
:101C8000D4C00E94F823D1C08B818230E1F078F477
:101C9000813009F0CAC080916A02FFEF8F9FC001B6
:101CA00011246FEF70E00E946D266C83BEC08330FC
:101CB00091F0843009F0B9C0809168028C838091E2
:101CC00069028D83B2C08091670280FF02C0869551
:101CD00004C080E002C080916B028C83A6C060913A
:101CE0006702709168028091690290916A020E9475
:101CF0000D239BC080E152C083E08A838AE58B83F9
:101D000094C0EA80FB80FE24EF24FE248C80912C7A
:101D10003801C7018A559F4F9301201B310B2815AD
:101D2000390508F082C02AE5E21623E0F20630F415
:101D30000E94B625D30114968C9302C0F30114823D
:101D4000FFEFEF1AFF0A2FEF621A720AE2CFEA8062
:101D5000FB80FE24EF24FE248C80912C3801C701E7
:101D60008A559F4F9301201B310B2815390508F028
:101D70005CC03AE5E31633E0F30628F4D301149689
:101D80006C910E94CA25BFEFEB1AFB0AEFEF6E1AA7
:101D90007E0AE5CF0E94601E48C084E08A8345C069
:101DA000EA80FB80FE24EF24FE248C80912C3801F5
:101DB000C70186969301201B310B28153905A8F51C
:101DC000F0E8EF16F10430F40E94B625D301149622
:101DD0008C9302C0F3011482FFEFEF1AFF0A2FEF7A
:101DE000621A720AE5CFEA80FB80FE24EF24FE240B
:101DF0008C80912C3801C70186969301201B310BF2
:101E00002815390590F430E8E316F10428F4D301DD
:101E100014966C910E94CA25BFEFEB1AFB0AEFEFF4
:101E20006E1A7E0AE8CF8FEF898340E250E0B80156
:101E300082E00E949814E0CBE9BCF9BC09B400FE32
:101E4000FDCF8091D8008F7D8093D8008091E000F5
:101E500082608093E0008091E00081FDFCCF0E94D1
:101E60005D20D3CB85E290E00E94B6251B821C82C8
:101E70001D82B6CE2B30310508F04DCD8BCD2B30E9
:101E8000310508F0A0CDDECD8091D30187FF11C0D0
:101E90008091E80082FD05C08091D1018111F8CFC9
:101EA00011C08091E8008B770BC08091D10188230D
:101EB00049F08091E80080FFF8CF8091E8008E77AC
:101EC0008093E8000895982F973068F59093E90083
:101ED000981739F07091EC002091ED005091F000CE
:101EE00003C0242F762F50E021FD02C09F5FECCF6E
:101EF0003091EB003E7F3093EB003091ED003D7F61
:101F00003093ED003091EB0031603093EB00709333
:101F1000EC002093ED005093F0002091EE0027FD9F
:101F2000E5CF80E008958F708093E90081E0089507
:101F30002091D9013091DA012617370748F0611551
:101F4000710539F42091E8002E772093E80001C054
:101F5000B901FC0120E06115710579F18091D10191
:101F60008823F1F18530F1F18091E80083FD3CC0D8
:101F70008091E80082FD2EC08091E80080FFEBCFC9
:101F80002091F3008091F20090E0922B6115710591
:101F900051F08830910538F421912093F10061507F
:101FA00071090196F3CF21E0089709F020E08091B4
:101FB000E8008E778093E800CECF2111CFCF0AC002
:101FC0008091D101882361F0853061F08091E80033
:101FD00083FD0AC08091E80082FFF2CF80E008957F
:101FE00082E0089583E0089581E008958091AE0134
:101FF00008958091DB01982F9670963011F48860D7
:1020000001C0877F0E9407200895AAE2B0E0EBE0BC
:10201000F0E10C94C026E3EDF1E08BED91E020912E
:10202000F10021938E179F07D1F78091D40183305F
:1020300009F463C030F4813071F0823009F49DC03E
:10204000B4C08A3009F489C08B3009F46EC089307D
:1020500009F0ABC020C08091D301813A09F0A5C03E
:102060008091E800877F8093E8008091D70190916C
:10207000D801892B21F460E28FEA91E003C060E08F
:1020800080E090E070E00E94980F8091E8008B77EC
:102090008093E8008AC08091D301813209F085C025
:1020A0008091D7019091D801009719F0029709F01B
:1020B0007CC08091E800877F8093E8008091E800F1
:1020C00082FD05C08091D1018111F8CF6EC02091B1
:1020D000F3008091F20090E0922B029731F480910E
:1020E000F100813011F0863021F48091F10080936D
:1020F000AE018091E8008B7754C08091D301813A82
:1021000009F053C08091D7019091D801892B09F033
:102110004CC08091E800877F8093E8008091E800C0
:1021200080FFFCCF80910C0137C08091D3018132B8
:10213000E1F58091D7019091D801892BB1F580917B
:10214000E800877F8093E8000E94440F8091D501CA
:1021500080930C010E945D2028C08091D3018132C0
:1021600021F58091E800877F8093E8000E94440F6A
:102170008091D6018093AD0118C08091D301813A3E
:10218000A1F48091E800877F8093E8008091E800C7
:1021900080FFFCCF8091AD018093F1008091E80039
:1021A0008E778093E8000E94440F8091E80083FFBF
:1021B000DFC18091D3019091D401492F50E04A3082
:1021C000510508F0D5C1FA01ED54FF4F0C94952646
:1021D000803821F0823809F0CBC108C08091CF014E
:1021E0009091D001992389F082600FC08091D7012E
:1021F0008F70873008F0BCC18093E9008091EB00BC
:1022000085FB882780F91092E9009091E800977F7C
:102210009093E8008093F1001092F10070C1282F94
:102220002D7F09F0A5C1882319F0823061F0A0C18B
:102230008091D501813009F09BC1933009F080E095
:102240008093D0012EC08091D50181112AC0809148
:10225000D7018F702FEF280F263008F089C18093A7
:10226000E9002091EB0020FF1CC0933021F4809105
:10227000EB00806214C09091EB0090619093EB00B2
:1022800021E030E0A90102C0440F551F8A95E2F712
:102290004093EA001092EA008091EB0088608093FE
:1022A000EB001092E9008091E800877F8093E800BE
:1022B0000E94440F5DC181115BC11091D5011F7750
:1022C0008091E3008078812B8093E3008091E80087
:1022D000877F8093E8000E94440F8091E80080FF90
:1022E000FCCF8091E30080688093E300111102C06D
:1022F00082E001C083E08093D1013AC180588230EE
:1023000008F036C12091D5013091D6012C3D53E023
:10231000350779F583E08A838AE289834FB7F89499
:10232000DE01139620E03EE051E2E32FF0E050930F
:102330005700E49120FF03C0E295EF703F5FEF701C
:102340008E2F90E0EA3010F0C79601C0C0968D93B2
:102350009D932F5F243149F74FBF8091E800877F1D
:102360008093E8006AE270E0CE0101960E94980F27
:10237000B4C08091D7019091D801432F55274330A5
:102380005105A9F068F44130510509F400C142300B
:10239000510509F0EDC08BE590E0E7E5F3E04BC0B7
:1023A0004132510529F14232510589F1E1C0C9019B
:1023B000992781309105A1F058F0029709F0D8C013
:1023C000E4ECF3E0E4918E2F90E0E4ECF3E030C035
:1023D000E4EFF3E0E4918E2F90E0E4EFF3E028C027
:1023E000E6EDF3E0E4918E2F90E0E6EDF3E020C01F
:1023F0008330910508F0BCC0880F991FFC01E45D93
:10240000FE4F0190F081E02D89E090E014C0833010
:10241000910508F0ADC0FC01EE0FFF1FEA5DFE4F15
:102420000190F081E02DDC01AD5DBE4F8C9190E01C
:10243000009709F49DC02091E800277F2093E800D1
:102440002091D9013091DA012817390708F4C90120
:1024500040E0009789F12091D101222309F43DC089
:102460002530D9F12091E80023FD37C02091E80004
:1024700022FD2FC02091E80020FFEBCF4091F30018
:102480002091F20030E0342B009759F028303105CC
:1024900040F444914093F100319601972F5F3F4FF4
:1024A000F3CF41E02830310509F040E02091E80009
:1024B0002E772093E800CDCF4111CDCF0AC0809177
:1024C000D101882351F0853041F08091E80083FDEF
:1024D00004C08091E80082FFF2CF8091E8008B7702
:1024E0008093E80045C0803809F042C08091E80040
:1024F000877F8093E8008091D2018093F1008091E2
:10250000E8008E77D3CE811133C08091D5019091B0
:10251000D6019927029764F58091E800877F809320
:10252000E8001091D5011093D2010E94440F1111BF
:1025300006C08091E30087FD02C081E001C084E015
:102540008093D10142E061EC81E00E94630F42E29E
:1025500061EC84E00E94630F42E261EC82E00E9441
:10256000630F42E260EC83E00E94630F8091D1012F
:102570008091E80083FF10C08091E800877F8093FE
:10258000E8008091EB0080628093EB0005C082E15F
:1025900090E0E2EBF3E04FCFAA96E3E00C94DC2668
:1025A0001F920F920FB60F9211242F933F934F93C8
:1025B0005F936F937F938F939F93AF93BF93CF93CB
:1025C000DF93EF93FF93C091E900CF708091EC000F
:1025D000D82FD17080FDD0E81092E9008091F000F2
:1025E000877F8093F00078940E9405101092E90094
:1025F0008091F00088608093F000CD2BCF70C09365
:10260000E900FF91EF91DF91CF91BF91AF919F9141
:102610008F917F916F915F914F913F912F910F908B
:102620000FBE0F901F901895E8EDF0E080818E7F2F
:1026300080831092E2001092DA001092E100A0EE86
:10264000B0E08C9181608C9380818F77808319BCFE
:10265000A7EDB0E08C918E7F8C9380818F7E8083FC
:102660001092AC010895A0E0B0E0E9E3F3E10C942E
:10267000BB26C8EDD0E088818F7E8883E7EDF0E04F
:1026800080818160808384E082BF81E08093AC019F
:1026900088818E7F888302EE10E0F801108210920C
:1026A000DA0081EEC82ED12CF601108288818F7756
:1026B000888388818068888388818F7D888319BC1E
:1026C0001092D1011092D2011092D0011092CF013C
:1026D00090EEE92EF12CF70180818B7F8083888139
:1026E0008160888342E060E080E00E94630FF60131
:1026F00080818E7F8083F8018081816080838081EA
:1027000088608083F70180818E7F808388818061EB
:102710008883CDB7DEB7E8E00C94D7261F920F92DE
:102720000FB60F9211242F933F934F935F936F93A4
:102730007F938F939F93AF93BF93EF93FF9380917A
:10274000E10082FF09C08091E20082FF05C0809114
:10275000E1008B7F8093E1008091DA0080FF2AC046
:102760008091D80080FF26C08091DA008E7F809310
:10277000DA008091D90080FF18C080E189BD82E134
:1027800089BD09B400FEFDCF81E08093D101809125
:10279000AC0181110FC00E9414130E943313809169
:1027A000E20084608093E20005C019BC1092D10160
:1027B0001092AC018091E10080FF17C08091E2008F
:1027C00080FF13C08091E2008E7F8093E2008091B1
:1027D000E20080618093E2008091D8008062809363
:1027E000D80019BC85E08093D1018091E10084FF7D
:1027F00030C08091E20084FF2CC080E189BD82E17D
:1028000089BD09B400FEFDCF8091D8008F7D8093F3
:10281000D8008091E1008F7E8093E1008091E200FA
:102820008F7E8093E2008091E20081608093E200DD
:102830008091D201882311F084E007C08091E300E9
:1028400087FD02C081E001C083E08093D1018091C7
:10285000D1018091E10083FF27C08091E20083FFD6
:1028600023C08091E100877F8093E10082E0809324
:10287000D1011092D2018091E1008E7F8093E1001E
:102880008091E2008E7F8093E2008091E20080617F
:102890008093E20042E060E080E00E94630F80915C
:1028A000F00088608093F000FF91EF91BF91AF91AD
:1028B0009F918F917F916F915F914F913F912F9158
:1028C0000F900FBE0F901F9018952091E40030914B
:1028D000E50095E64091EC00842F817040FF23C015
:1028E0008091E80080FD1DC08091D101882399F07E
:1028F000853099F08091EB0085FD11C04091E40096
:102900005091E5002417350729F3915011F09A01F1
:10291000E1CF84E0089582E0089583E0089581E0A6
:10292000089580E008954091E80042FFDDCF0895CA
:102930000F931F93CF93DF938B01EA019091D10105
:10294000943079F58F708093E9008FEF9091E800D3
:10295000815095FD06C095ED9A95F1F70000811123
:10296000F5CF8091E80085FF1CC00E946514882384
:1029700061F08091E8008E778093E80012C0F80142
:1029800081918F018093F1002197209791F380919D
:10299000E80085FDF4CF8091E8008E778093E80011
:1029A000E4CFDF91CF911F910F91089543E050E064
:1029B000BC0184E00E949814089546E050E0BC01F8
:1029C00084E00E9498140895CF93DF93EC018091E6
:1029D0000C01811105C048E050E0BE0181E00BC050
:1029E0008091AA0187FF03C040E284E002C048E072
:1029F00081E050E0BE010E94981480E2FE01AFEA3F
:102A0000B1E001900D928A95E1F7DF91CF910895A1
:102A100087E797E790930108809300089AE088E1A0
:102A20000FB6F894A895809360000FBE9093600055
:102A3000FFCF78941F920F920FB60F9211248F93AD
:102A40009F93AF93BF938091A6019091A701A0910E
:102A5000A801B091A9010196A11DB11D8093A60105
:102A60009093A701A093A801B093A901BF91AF9142
:102A70009F918F910F900FBE0F901F9018959C0102
:102A80004FB7F8948091A6019091A701A091A80159
:102A9000B091A9014FBF821B930B089580E0089568
:102AA0009091AA0192FF0DC0282F2871283019F4A7
:102AB000877F846006C0282F2471243011F48B7F17
:102AC000886093FF0DC0282F2871283119F4877E64
:102AD000846106C0282F2471243111F48B7E886113
:102AE0002091AB0120FF0DC0382F3871383019F418
:102AF000877F816006C0382F3171313011F48E7FAD
:102B0000886021FF0DC0282F2871283119F4877E95
:102B1000816106C0282F2171213111F48E7E8861D8
:102B200094FD877E0895F894E82FE295EF70F0E029
:102B300031A1282F2F7081E090E001C0880F2A95E5
:102B4000EAF7982F9095932391A392A1892B82A3C2
:102B500078940895A4E0B0E0E0EBF5E10C94B82699
:102B600019821A821B821C820BE111E0AE014F5FB9
:102B70005F4F7A015A01CC24C394D12CF801808193
:102B80008F3F09F441C0F894E82FE295EF70F0E030
:102B900021A18F70A60102C0440F551F8A95E2F74C
:102BA000CA01922F982B91A392A18095892382A389
:102BB000789400C0EFE1F1E0912C31E021912F3FBA
:102BC00089F0A22FA295AF70B0E090968C9190E022
:102BD0002F7002C0959587952A95E2F780FD02C077
:102BE000832F01C080E0982A330F51E0E332F507CC
:102BF00029F7F80180818F3F11F00E949315F0EAC8
:102C0000FA95F1F7F70190820F5F1F4FFFEFEF1A70
:102C1000FF0A41E00F31140709F0B0CF44E050E063
:102C2000B50185E991E00E94F526892BA9F08981FB
:102C30009A81AB81BC818093950190939601A0937A
:102C40009701B093980181E080935B020E940E1D72
:102C500090935A028093590280915B02811102C0C5
:102C600080E027C08091590290915A020E943F153E
:102C70000597B0F344E050E065E971E082EA91E045
:102C80000E94F526892B91F08091950190919601F3
:102C9000A0919701B09198018093A2019093A30114
:102CA000A093A401B093A50181E001C080E010923F
:102CB0005B022496EBE00C94D426743048F4643024
:102CC00038F4843028F4462F672F0E94CC1E0895D4
:102CD00080E090E00895CF93DF938238910569F109
:102CE000B0F48133910509F477C048F48932910535
:102CF00009F469C08A32910509F473C092C0853322
:102D0000910509F45BC089339105B9F08AC0833E0F
:102D1000910591F138F4803E9105D1F0823E910504
:102D200031F17FC0863E9105D9F1873E9105E9F1E9
:102D3000843E910509F075C028C02091AA0120FDAC
:102D40005BC021FD59C02091AB0123FD61C069C06A
:102D50008091AA0180FD4AC08091AB0180FF4CC0E8
:102D60008091AA0184FD50C183EE90E04FC1809113
:102D7000AA0182FF3EC0F4CF8091AA0182FD39C032
:102D80008091AB0180FD38C0EBCF8091AB0181FF1A
:102D900039C08091AA0184FD37C187EE90E036C129
:102DA0008091AA0183FF2BC0F4CF8091AA0183FDFB
:102DB00026C08091AB0181FD25C0EBCF8091AA0197
:102DC00085FD26C022C08091AA0185FD1EC080918C
:102DD000AB0183FF1DC00AC08091AA0186FD1BC004
:102DE0001DC08091AA0186FD19C015C089E390E03D
:102DF0000DC182EE90E00AC180EE90E007C186EE40
:102E000090E004C184EE90E001C185E390E0FEC053
:102E100089E290E0FBC08AE290E0F8C081E390E0B4
:102E2000F5C0EC01811530E5930708F053C081151A
:102E300060E4960720F0CE019F70906AE7C0803E64
:102E4000910588F58D3C910518F0CE019065DEC0A6
:102E5000883A9105C0F4853A910550F08C2F855A37
:102E6000C82FD0E0CE5CDE4F888190E09064CEC069
:102E70008130910509F4C5C008F4C6C0049708F470
:102E8000C3C0CE01C3C0813C910508F0BDC08C2FEA
:102E9000885AC82FD0E0CC0FDD1FCB5CDE4F888175
:102EA00099819464B3C08115904258F08D2F8F7131
:102EB0000E945015282F2F71CE0199279062922BD6
:102EC000A5C0C11581E0D807E0F6C83ED10508F0DD
:102ED0009BC0D7CFC03692E5D90708F053C0C034A5
:102EE00022E5D207B8F08C2F8F718695869570E217
:102EF000879FA00111248C2F837021E030E0B9015D
:102F000002C0660F771F8A95E2F7CB019C68842B7D
:102F1000952B7CC0C03232E5D30740F08C2F8F71E7
:102F200090E0982F8827816F906A70C0C11562E584
:102F3000D607B0F08C2F8695869520E2829FA0015F
:102F400011248C2F837021E030E0B90102C0660F9C
:102F5000771F8A95E2F7CB01842B952B9D6856C08D
:102F60008C2F8F710E94501595E0D695C7959A9534
:102F7000E1F7CF70D0E0DC2FCC27D0699E01282B61
:102F8000C90144C0C03A72E5D70708F58C2F8F718C
:102F9000C03892E5D907A8F48695869570E2879F98
:102FA000900111248C2F837041E050E0BA0102C0DF
:102FB000660F771F8A95E2F7CB019A68822B932BD5
:102FC00025C090E0982F8827846F906A1FC0C03C6E
:102FD00022E5D20750F48C2F8F710E9450158F710B
:102FE00090E0982F8827906211C0C03E32E5D30749
:102FF00058F4CE018F719927982F8827806F906A97
:1030000005C081E090E002C080E090E0DF91CF91C8
:10301000089580E090E00E94C425873E9E4F19F4F9
:103020000E942E1F089580E0089567EE7EEF80E0F5
:1030300090E00E94E82560E082E090E00E94CA25CE
:1030400060E083E090E00E94CA251092580260E0A0
:1030500074E184E090E00E94E82560E086E090E082
:103060000E94CA256FEF87E090E00E94CA2540E0E9
:1030700050E0BA0188E090E00E94DC2560E08DE03D
:1030800090E00E94CA2540E050E0BA0188E190E05B
:103090000E94DC2560E087E190E00E94CA2540E0C4
:1030A00050E0BA018CE190E00E94DC2560E070E025
:1030B00080E290E00E94E82540E050E0BA0188E11B
:1030C00090E00E94DC2580E00E94FF1E0E941E1FEF
:1030D00040E050E0BA018FE090E00E94DC2540E043
:1030E00050E0BA0183E190E00E94DC2508958091D0
:1030F00057028111109257020895809590915602BF
:10310000892380935602089590915602809155022A
:10311000982B9093DC01809157028823D9F0892B5A
:103120008093DC0180910C01882331F08091AA0109
:1031300087FF02C08EE101C086E0EEEDF1E090E095
:10314000815028F021912223D9F39F5FF9CF91116B
:103150000E94771840E250E065E372E08CED91E068
:103160000E94F526892B21F180E2ECEDF1E0A5E348
:10317000B2E001900D928A95E1F7E0917102F09131
:1031800072023097A9F080910C01882359F0809148
:10319000AA0187FF07C08091DC018093DD0186E0F2
:1031A0008093DC010280F381E02D8CED91E00995A4
:1031B0000895209134028095822380933402982FC1
:1031C000977099F430E0482F082E000C550B241707
:1031D000350759F09091AB0192FF07C08595859511
:1031E00085950E940A201092340208959091AB01B7
:1031F00092FB222720F9281779F080FB92F990930F
:10320000AB016091AA017091AB0184E090E00E9453
:10321000E82582E00E94D9180895809133029091A8
:103220000202891719F08F5F8770FBCF08950F9303
:103230001F93CF93DF938091010282958F7009F0E5
:103240005AC08091FE01882309F455C08091330251
:10325000109102026091FC017091FD01C091FF018B
:10326000D091000291E06F3F09F090E0292F06E035
:10327000811709F440C0209721F07F3F21F030E012
:1032800003C031E001C0322F90E030FD31C0089F13
:10329000F001099FF00D1124DF01AD5FBD4F1196C4
:1032A0003C911197371324C03C91361321C01296DC
:1032B0003C91129731111CC013964D915C9114975B
:1032C0004C1B5D0B483C510598F4809101028F70B6
:1032D000806180930102E85FFD4F80818F70806183
:1032E00080838CEF91E00E941D040E940D1903C0A1
:1032F00001968770BDCFDF91CF911F910F910895F7
:10330000A1E1B0E0E6E8F9E10C94B8268C0185E093
:10331000F801DE011D9601900D928A95E1F7F80102
:10332000E2809091FC016091FD014091FF0150917C
:1033300000024115510531F06F3F31F481E09F3FAC
:1033400019F403C081E001C080E0F82FF1709F2ED6
:1033500080FD1BC1F80130812181C380D4808CEFB6
:10336000A82E81E0B82EF090FE01F601E41BF50BCB
:10337000FF2009F4C7C080910102E83CF10508F084
:1033800092C0482F407F09F051C0621311C09313BF
:103390000FC0FE2CE1100CC08F7080618093010281
:1033A000C5010E941D0480910102F80185832AC194
:1033B000C114D10431F02F3F31F481E03F3F19F4C3
:1033C00003C081E001C080E080FD03C081E08E2564
:1033D00002C080E090E0F82FF170FF2E80FF1CC04B
:1033E000809133024091020256E0841709F4E8C04C
:1033F00090E0589FF001599FF00D1124ED5FFD4FB3
:103400006181261306C06081631303C06281E612E6
:1034100003C001968770E9CFFE2CEE2009F4F2C0BC
:103420008091010281608093010249C0621306C04D
:10343000931304C0E11002C0F80186C0C8010E94C5
:103440002620882351F1EE2041F120910102822FA4
:1034500082958F7090E0029774F08091FC019091BA
:10346000FD0198878F831986DB86CA862C87CE015B
:1034700007960E941D0486E0F801ACEFB1E00190D0
:103480000D928A95E1F70E9417190AC06217C9F0D8
:10349000C8010E94262081111EC0C8010E941D047F
:1034A000FF24F394AFC0482F407F81F78CEF91E069
:1034B0000E941D0486E0F50111928A95E9F7F12C2E
:1034C000A1C09313E5CFE110E3CFF8018583C801D4
:1034D0000E941D0454C0EE2001F320910102822FAE
:1034E00082958F7090E0029734F28091FC01909168
:1034F000FD019A8389831B82DD82CC822E83CE01DB
:103500000196B7CFE83CF105D0F5FE2CEE2029F26C
:10351000621327C0931325C02091010220FD18C01B
:10352000822F82958F70482F50E04115510581F010
:10353000F80125834F30510541F08F5F982F929508
:10354000907F822F8F70892B8583C8010E941D0474
:1035500086E0F801ACEFB1E001900D928A95E1F7B9
:1035600051C0C8010E942620811185CF809101029F
:10357000816080930102C8010E941D0443C086E05F
:10358000F50111928A95E9F73DC0EE2009F485CF47
:10359000C8010E942620F82E882309F47ECF86E0F9
:1035A000F801ACEFB1E001900D928A95E1F78091BE
:1035B000FC019091FD010E94911F0E94171922C0E9
:1035C0003D872E878D859E850E94911F292F2295EC
:1035D0002F70223028F49F7039F0811105C00BC084
:1035E000243028F49F7049F4805E883020F0C801B0
:1035F0000E941D049F2CF92C05C0F8019581907F35
:1036000099F7F9CF8F2D6196EBE00C94D4260895AD
:10361000CF93FC01C281848191E09483E8EFF3E0D1
:103620003491E7E7F4E02491C33040F490916802CC
:10363000909362029091690290936302811105C098
:10364000109265021092640260C080916502882326
:1036500021F18150809365024FEF849FC0011124B6
:103660006091660270E00E946D26FB01FF27E85022
:10367000FC4F8491E82FE31B4FEFE49FC00111241E
:10368000231B622F70E00E946D2680916A02689F62
:10369000B00111247093640238C00E94A6252091C5
:1036A0006A022695215830E0A901440F551F322F98
:1036B0002227240F351F232F3327821793072CF53A
:1036C000C330A0F00E94A6256FEF70E00E94812613
:1036D000809362020E94A625209169022695622F9E
:1036E00070E00E948126280F2093630210926402EA
:1036F00080916A02843120F0893C18F088EC01C086
:1037000084E180936602809365022FE532E0409168
:10371000640260916302809162020E9454230E94BD
:10372000BC22CF910895CF93DF93EC018C812FE5DC
:1037300032E0882311F040E002C040916A026091BB
:103740006902809168020E9454230E94BC228C81ED
:1037500090E00196817099278C83DF91CF91089535
:10376000A0E0B0E0E6EBFBE10C94B726EC014C8165
:10377000042F10E09801D8010E9452269B01AC0151
:103780000E941D266B017C01E0E2F0E0E01BF10BE2
:10379000A5E5B0E09B01AC010E941D264B015C0138
:1037A0009F01DF010E94A2269B01AC010E942826F6
:1037B0009B01AC012C0D3D1D4E1D5F1DC501B401CB
:1037C0000E943026922F2A3228F483E0289FA001FD
:1037D00011240DC045E550E0491B51099A01220F03
:1037E000331F420F531F57FF02C04F5F5F4F559566
:1037F000479540952FE532E06091690285E5891B88
:103800000E9454230E94BC228C81811102C091E04D
:1038100003C0803219F49FEF90930F0190910F0134
:10382000890F8C83CDB7DEB7ECE00C94D3261092D1
:10383000600210925F021092610280915D02181680
:1038400074F080910E0187FD0AC02FE532E04091AF
:103850006A0260916902809168020E9454230E946A
:10386000BC2280910D0190915D02980F90935D02B2
:1038700020910E01280F20930E01121614F497FDCB
:1038800003C0819580930D0108950F931F93CF93EB
:10389000DF93FC01828180FF02C01FEF01C011E0B5
:1038A0001092600210925F0210926102C4E0D0E0B8
:1038B00000E080915C02800F823024F487FD8F5FEE
:1038C000811113C080916A028C9FA0018D9F500DC1
:1038D000112455954795559547952FE532E0609110
:1038E0006902809168020E945423010F219709F711
:1038F0000E94BC22113041F480915C02882331F097
:10390000815080935C0202C010925C02DF91CF91E3
:103910001F910F910895CF93DF93EC012FE532E0D3
:1039200040916A02609169028C810E9454230E9436
:10393000BC229A818C8190FF02C08F5F01C08150B0
:103940008C83DF91CF910895A3E0B0E0EAEAFCE137
:103950000C94BF268C0180915E0281110AC09E01E9
:103960002F5F3F4F4FEF6FEF0E9454238A81809368
:103970005E02F8018481813051F028F0823061F4D8
:1039800040915E020AC080915E0240E007C06091F3
:103990005E0240E080E003C040E080E060E00E9422
:1039A000ED22F801848190E0019663E070E00E94CE
:1039B000812684832396E4E00C94DB26CF93DF9367
:1039C000EC01E7E6F2E0438162818C810E94E02312
:1039D0008C818F5F8C83DF91CF910895CF93DF939C
:1039E000EC01EC81F0E0E850FC4F4491E7E6F2E0B6
:1039F000628181810E94E0238C818F5F8C83DF91C3
:103A0000CF9108952FB7F8946091A6017091A70106
:103A10008091A8019091A9012FBF08952FB7F89424
:103A20008091A6019091A701A091A801B091A90150
:103A30002FBF08951F920F920FB60F9211248F93EC
:103A40009F93AF93BF9380917502811113C08091B2
:103A5000A6019091A701A091A801B091A90141965A
:103A6000A11DB11D8093A6019093A701A093A80169
:103A7000B093A901BF91AF919F918F910F900FBE0D
:103A80000F901F90189520910C012223C9F02091CE
:103A9000AA0127FF15C0262F2695269526952E319B
:103AA000C8F4FC01E20FF11D677081E090E001C0F5
:103AB000880F6A95EAF78095928189238283089519
:103AC000FC0106962281621301C012823196E8172A
:103AD000F907C1F7089520910C012223C1F020912C
:103AE000AA0127FF14C0262F2695269526952E314C
:103AF00030F5FC01E20FF11D677081E090E001C03C
:103B0000880F6A95EAF79281892B82830895FC01D8
:103B100032962FEF30E04191641789F02F3F19F46E
:103B2000411101C0232F3F5F3630A9F72F3F39F0F5
:103B3000FC01E20FF11D27FDFA95628308950895B7
:103B4000A3E0B0E0E6EAFDE10C94C1262091730207
:103B50003091740228173907A1F090937402809372
:103B60007302E0917102F0917202309751F024E0FB
:103B700029839B838A830680F781E02DCE010196FD
:103B800009952396E2E00C94DD26A3E0B0E0EBEC8F
:103B9000FDE10C94C12620916F023091700228172C
:103BA0003907A1F09093700280936F02E091710247
:103BB000F0917202309751F023E029839B838A832E
:103BC0000680F781E02DCE01019609952396E2E06B
:103BD0000C94DD26E0917102F0917202309729F089
:103BE0000190F081E02D0995089580E008950F93EC
:103BF0001F93CF93DF93C42FD22FFC0182818823A0
:103C0000B1F040936E020E940E1D90936D0280935E
:103C10006C0280E28C0F883008F04DC0C77081E0E4
:103C200001C0880FCA95EAF70E94932044C0809192
:103C30006E02481330C080916C0290916D020E9418
:103C40003F15883C910538F510E21D0FCD17B9F0EE
:103C500080E28C0F883040F4C77081E001C0880F8B
:103C6000CA95EAF70E948C20183010F581E09D2F4C
:103C7000977001C0880F9A95EAF70E949320802FD1
:103C80000E949D221830B8F4D77081E001C0880FDF
:103C9000DA95EAF70AC080E28C0F883060F4C770CA
:103CA00081E001C0880FCA95EAF70E948C2003C00A
:103CB000802F0E949D22DF91CF911F910F91089537
:103CC000CF93DF93C6EAD0E060E0CE010E94CA2520
:103CD0002196C11584E0D807B9F7DF91CF910895F7
:103CE0001F93CF93DF93962F8430E8F46430D8F499
:103CF0004430C8F4632F122FC42FD0E0CC0FDD1F47
:103D000028E0929FC00DD11D112490E2899FC00D23
:103D1000D11D1124CE0186960E94CA25612FCE01A5
:103D200087960E94CA25DF91CF911F910895A0E048
:103D3000B0E0EDE9FEE10C94B926A12CE12CF12CC8
:103D4000B12C00E010E0C0E0D0E06701C00ED11E51
:103D5000F601EC0FFD1FEE0FFF1FE850FB4F259102
:103D600034914C2F6B2D8A2D0E94701E2196C430E9
:103D7000D10571F70C5F1F4FB39484E0B812E3CF05
:103D800080E1E80EF11CA39484E0A812D9CFCDB74E
:103D9000DEB7EAE00C94D5260F931F93CF93DF9301
:103DA000843008F56430F8F44430E8F4C42FD0E0EF
:103DB000CC0FDD1F28E0629FC00DD11D112430E221
:103DC000839FC00DD11D1124CE0186960E94B62579
:103DD00090E0182F0027CE0187960E94B625980103
:103DE000282BC90102C080E090E0DF91CF911F91A4
:103DF0000F91089585E290E00E94CA250895CF931F
:103E0000C82F811102C06FEF01C062E282E290E030
:103E10000E94CA25C11102C06FEF01C062E183E2B6
:103E200090E00E94CA25C11102C06FEF01C068E096
:103E300084E290E00E94CA25CF91089580E00E941C
:103E4000FF1E60E070E0CB010E94FA1E0E94971EE8
:103E50000E94601E81E00E94FF1E089582E290E0B1
:103E60000E94B625823281F483E290E00E94B6255A
:103E7000823151F484E290E00E94B62591E08830CE
